:1000000094C0189501C018950FB617EE12BF7395DE
:1000100080FF0BC00894809B88944795783019F432
:10002000112719BF82600FBE1895713011F4919895
:10003000FACF7A3029F4919A112719BF8160F3CF52
:1000400040FD919A40FF91984695EDCF81E012E0F6
:1000500013BF899A889808958827772712E019BFD7
:1000600080FFFECF0895809BFECF8099FECF13EED8
:1000700012BF12E018BF19BF772781FFFECF8D7F17
:1000800008952FEF2A95F1F71A95D9F70895939AC5
:1000900018E0331F10F4C69A01C0C698C79A26E02C
:1000A0002A95F1F7C79823E02A95F1F71A9589F771
:1000B00093980895939A18E030E0330FB599316022
:1000C000C79A26E02A95F1F7C79823E02A95F1F719
:1000D0001A9599F79398089541E4BEDF46E5BCDF91
:1000E00042E5BADF40E2B8DF49E4B6DF43E5B4DF1A
:1000F00040E5B2DF089510E018BB1FED17BB0131DA
:1001000021F0013211F0C29A02C0C19A00C0C39A14
:100110001FEFB7DF1FEFB5DFC49A1FEFB2DFC49840
:100120001FEFAFDF1FEFADDF089510E01BBF1FEF24
:1001300012BB00008B9A939810E018BB1FED17BB01
:1001400085DF7894939AAAE01FEF9BDFAA95E1F7E9
:100150009398AAE01FEF95DFAA95E1F7939AAAE09A
:100160001FEF8FDFAA95E1F793987DDF4B31E9F31D
:10017000483711F4939A16C1493711F4939812C174
:10018000443519F470DF042F0DC1433511F4A4DF99
:10019000ECCF463529F443E35FDF45E35DDFE5CF90
:1001A000463729F443E358DF41E356DFDECF4037DB
:1001B00019F443E551DFD9CF013139F0023129F08B
:1001C000013219F0023209F0EAC0403529F593DF17
:1001D0003CEA5DDF33E55BDF0132B9F40232A9F0BE
:1001E000A0E268DF333599F030E051DFC79A26E0AE
:1001F0002A95F1F7C79823E02A95F1F73CEA47DF03
:1002000033E545DFAA9569F7CAC030E040DF30E04A
:100210003EDF10E136DFC6C0433481F424DF38E42A
:1002200036DF362F34DF352F32DF342F30DF10E268
:1002300028DF11E02227510F621FB4C0433661F45A
:1002400012DF30E424DF362F22DF352F20DF342F7A
:100250001EDF10E216DFA6C04235B9F438E217DF20
:10026000362F15DF352F13DF25DF432FF5DE30E284
:100270000EDF362F0CDF352F0ADF1CDF432FECDEBD
:1002800011E02227510F621F70CF413429F4EBDEB9
:10029000642FE9DE542F86C0443461F4E4DE30EC90
:1002A000F6DE362FF4DE352FF2DE342FF0DE10E2EC
:1002B000E8DE78C0443651F430EAE9DE362FE7DE76
:1002C000352FE5DEF7DE432FC7DE4FCF4C3429F460
:1002D00010E018BB10E017BB65C0453659F43CEA86
:1002E000D6DE30E8D4DE34E0D2DE30E0D0DE10E31B
:1002F000C8DE58C04C3671F4B6DE3CEAC8DE342F96
:100300003670306EC4DE30E0C2DE30E0C0DE10E3B6
:10031000B8DE48C0463671F4A6DE3CEAB8DE342FBB
:100320003170306AB4DE30E0B2DE30E0B0DE10E3CF
:10033000A8DE38C0463451F438E5A9DE30E0A7DE47
:1003400030E0A5DEB7DE432F87DE0FCF433789F4D9
:10035000B2E005D0B1E003D0B0E001D006CF30E389
:1003600096DE30E094DE3B2F92DEA4DE432F74DE77
:1003700008954A33A1F477DEC42F75DED42F73DEDF
:10038000E42F03D01FEF7DDE0DC03C2F80DE3D2F1C
:100390007EDE3E2F7CDE8EDE432F5EDE08954FE351
:0A03A0005BDEE3CE4DE058DEE0CE58
:00000001FF
